:100000000C9446000C9465000C9465000C946500FB
:100010000C9465000C9465000C9465000C946500CC
:100020000C9465000C9465000C9465000C946500BC
:100030000C9465000C9465000C9465000C946500AC
:100040000C9465000C9465000C9465000C9465009C
:100050000C9465000C9465000C9465000C9465008C
:100060000C9465000C9465000C9465000C9465007C
:100070000C9465000C9465000C9465000C9465006C
:100080000C9465000C9465000C94650011241FBE4F
:10009000CFEFD0E1DEBFCDBF12E0A0E0B1E0E2E201
:1000A000FFE100E00BBF02C007900D92AC36B10734
:1000B000D9F712E0ACE6B2E001C01D92AE38B1074C
:1000C000E1F70E9429020C948F0F0C9400008DED33
:1000D0008A95F1F70895AA9A9DED292F2A95F1F7AF
:1000E0008BBB892F8A95F1F7AC9A892F8A95F1F706
:1000F000AC989A95F1F70895AA989DED292F2A9525
:10010000F1F78BBB892F8A95F1F7AC9A892F8A95E5
:10011000F1F7AC989A95F1F70895AA989DED892F7B
:100120008A95F1F781E08BBB892F8A95F1F7AC9A1C
:10013000892F8A95F1F7AC989A95F1F708951BBA33
:100140008FEF8ABB15BA8CE384BBAB98AC98AA98A6
:100150009DED892F8A95F1F78BE38BBB892F8A95CB
:10016000F1F7AC9A892F8A95F1F7AC98892F8A9587
:10017000F1F7AA98892F8A95F1F78CE08BBB892F2C
:100180008A95F1F7AC9A892F8A95F1F7AC989A95F0
:10019000F1F70E948D000895823041F0833041F0E4
:1001A000813011F490E405C090E003C090E101C0FB
:1001B00090E5960F9068AA988DED282F2A95F1F773
:1001C0009BBB982F9A95F1F7AC9A982F9A95F1F7D7
:1001D000AC988A95F1F70895FC012DED11C0AA9A0B
:1001E000822F8A95F1F79BBB822F8A95F1F7AC9A03
:1001F000822F8A95F1F7AC98822F8A95F1F7319684
:100200009081992361F70895FC012DED11C0AA9A00
:10021000822F8A95F1F79BBB822F8A95F1F7AC9AD2
:10022000822F8A95F1F7AC98822F8A95F1F7319653
:100230009081992361F70895382F6AE00E944C0F4E
:10024000805DAA9A2DED922F9A95F1F78BBB822FA4
:100250008A95F1F7AC9A822F8A95F1F7AC98822FA4
:100260008A95F1F7832F0E944C0F905DAA9A822FF6
:100270008A95F1F79BBB822F8A95F1F7AC9A822F72
:100280008A95F1F7AC982A95F1F70895382F982FB1
:1002900092959F709A3010F4905D01C0995CAA9A73
:1002A0008DED282F2A95F1F79BBB982F9A95F1F7A2
:1002B000AC9A982F9A95F1F7AC988A95F1F7932F0D
:1002C0009F709A3010F4905D01C0995CAA9A8DEDF0
:1002D000282F2A95F1F79BBB982F9A95F1F7AC9AA6
:1002E000982F9A95F1F7AC988A95F1F708951F9396
:1002F000182F892F0E944601812F0E9446011F91CD
:1003000008952F923F924F925F926F927F928F92B9
:100310009F92AF92BF92CF92DF92EF92FF920F9394
:100320001F93CF93DF932C01A59AC0E0D0E03B014F
:10033000882477FC8094982C80E7282E81E0382E42
:1003400071C085B390E2892785BBC401B3010E94C7
:100350007A095B016C0122E539E44DE950E40E9421
:1003600046077B018C0120E030E040E85FE30E941B
:100370004A09882314F461E052C020E030E04FE7DE
:1003800053E4C801B7010E94EA0818160CF043C0F4
:1003900020E030E04AE754E4C601B5010E9440087D
:1003A0005B016C0126E636E646E655E40E94460708
:1003B0007B018C0120E030E040E85FE30E944A09C5
:1003C00088231CF461E070E022C020E03FEF4FE79B
:1003D00057E4C801B7010E94EA081816A4F420E007
:1003E00030E040E251E4C601B5010E9446070E9498
:1003F000700505C0C1010197F1F7615070406115AA
:100400007105C1F70EC0C801B7010E947005CB018C
:100410000197F1F706C0C801B7010E9470056A95FF
:10042000F1F72196C415D5050CF48BCFDF91CF9150
:100430001F910F91FF90EF90DF90CF90BF90AF9002
:100440009F908F907F906F905F904F903F902F90F4
:1004500008952F923F924F925F926F927F928F9268
:100460009F92AF92BF92CF92DF92EF92FF920F9343
:100470001F93DF93CF930F92CDB7DEB70E949F00FB
:100480000E948D008CEC9CE10197F1F760E080E028
:100490000E94CC0080E091E00E94EC0060E081E0EE
:1004A0000E94CC0080E191E00E94EC0060E271E0EB
:1004B00083E892E00E94A30C10928D028FEF80934C
:1004C00063019AB39983909388026091600170915F
:1004D000610180E090E00E942C0A1B012C0122E5C2
:1004E00039E44DE950E40E9446075B016C0120E0CD
:1004F00030E040E85FE30E944A09882314F461E099
:1005000053C020E030E04FE753E4C601B5010E943C
:10051000EA0818160CF044C020E030E04AE754E442
:10052000C201B1010E9440083B014C0126E636E6BB
:1005300046E655E40E9446077B018C0120E030E04E
:1005400040E85FE30E944A0988231CF461E070E000
:1005500023C020E03FEF4FE757E4C801B7010E94F6
:10056000EA081816ACF420E030E040E251E4C4019F
:10057000B3010E9446070E94700506C080E791E023
:100580000197F1F76150704061157105B9F70EC020
:10059000C801B7010E947005CB010197F1F706C0B1
:1005A000C601B5010E9470056A95F1F7D09AD19AFB
:1005B000D29AD39AD498D598D698D798EEE0EBBB38
:1005C00020E030E040E85FE3C601B5010E944A093F
:1005D000882314F461E053C020E030E04FE753E497
:1005E000C601B5010E94EA0818160CF044C020E0CC
:1005F00030E04AE754E4C201B1010E9440083B01E7
:100600004C0126E636E646E655E40E9446077B01A5
:100610008C0120E030E040E85FE30E944A09882333
:100620001CF461E070E023C020E03FEF4FE757E4A7
:10063000C801B7010E94EA081816ACF420E030E0C7
:1006400040E251E4C401B3010E9446070E947005D4
:1006500006C080E791E00197F1F7615070406115A5
:100660007105B9F70EC0C801B7010E947005CB0132
:100670000197F1F706C0C601B5010E9470056A95A1
:10068000F1F7CC9903C0F1E0F0936301CD9903C079
:1006900084E080936301CE9903C097E09093630157
:1006A000CF9903C0E4E6E0936301FDE0FBBB20E0EB
:1006B00030E040E85FE3C601B5010E944A098823A3
:1006C00014F461E053C020E030E04FE753E4C6018A
:1006D000B5010E94EA0818160CF044C020E030E092
:1006E0004AE754E4C201B1010E9440083B014C01B9
:1006F00026E636E646E655E40E9446077B018C0175
:1007000020E030E040E85FE30E944A0988231CF4BF
:1007100061E070E023C020E03FEF4FE757E4C801FD
:10072000B7010E94EA081816ACF420E030E040E27D
:1007300051E4C401B3010E9446070E94700506C03F
:1007400080E791E00197F1F7615070406115710504
:10075000B9F70EC0C801B7010E947005CB0101971F
:10076000F1F706C0C601B5010E9470056A95F1F760
:10077000CC9903C082E080936301CD9903C095E0DA
:1007800090936301CE9903C0E8E0E0936301CF99B1
:1007900002C010926301FBE0FBBB20E030E040E8C8
:1007A0005FE3C601B5010E944A09882314F461E0A1
:1007B00053C020E030E04FE753E4C601B5010E948A
:1007C000EA0818160CF044C020E030E04AE754E490
:1007D000C201B1010E9440083B014C0126E636E609
:1007E00046E655E40E9446077B018C0120E030E09C
:1007F00040E85FE30E944A0988231CF461E070E04E
:1008000023C020E03FEF4FE757E4C801B7010E9443
:10081000EA081816ACF420E030E040E251E4C401EC
:10082000B3010E9446070E94700506C080E791E070
:100830000197F1F76150704061157105B9F70EC06D
:10084000C801B7010E947005CB010197F1F706C0FE
:10085000C601B5010E9470056A95F1F7CC9903C0F5
:1008600083E080936301CD9903C096E09093630188
:10087000CE9903C0E9E0E0936301CF9903C085E618
:1008800080936301F7E0FBBB20E030E040E85FE3EA
:10089000C601B5010E944A09882314F461E053C0DF
:1008A00020E030E04FE753E4C601B5010E94EA08BA
:1008B00018160CF044C020E030E04AE754E4C201CE
:1008C000B1010E9440085B016C0126E636E646E66F
:1008D00055E40E9446077B018C0120E030E040E8AF
:1008E0005FE30E944A0988231CF461E070E023C0A2
:1008F00020E03FEF4FE757E4C801B7010E94EA0844
:100900001816ACF420E030E040E251E4C601B50135
:100910000E9446070E94700506C080E791E001979B
:10092000F1F76150704061157105B9F70EC0C8014B
:10093000B7010E947005CB010197F1F706C0C6010F
:10094000B5010E9470056A95F1F7CC9903C08BE060
:1009500080936301CD9903C08CE080936301CE99AD
:1009600003C09DE090936301CF9903C0EEE0E09354
:1009700063018FE08BBBF981FABB90916301809199
:100980006201981709F45FC0909362019A3008F0F1
:100990005AC080916C02882341F460E081E00E949B
:1009A000CC0085E291E00E94EC0080916C028D5FAA
:1009B00080936C028D3058F060E081E00E94CC00A2
:1009C00085E291E00E94EC0082E080936C028091CD
:1009D000810290918202FC01E757FD4F2091630153
:1009E000205D208301969093820280938102049778
:1009F00021F4109282021092810260916C0281E0D7
:100A00000E94CC008091630190E09F938F93E6E376
:100A1000F1E0FF93EF938DE692E09F938F930E9416
:100A2000AA0C8DE692E00E94EC0068EE73E084E68A
:100A300090E00E948101EDB7FEB736960FB6F894AC
:100A4000FEBF0FBEEDBF80916301843609F036CD45
:100A500010926C02109282021092810260E081E09A
:100A60000E94CC0069E872E083E892E00E949A0C50
:100A7000009739F489E391E00E94EC0068EE73E09E
:100A800014C08AE491E00E94EC0064EF71E088E514
:100A900092E00E94810180ED97E0E0E7F1E031977C
:100AA000F1F70197D1F764EF71E088E592E00E94D9
:100AB000810180E197E2E0E7F1E03197F1F70197FA
:100AC000D1F760E081E00E94CC0085E291E00E94D5
:100AD000EC006BE571E089E892E00E94A30CEECC9B
:100AE000EF92FF920F931F937B018C0120E030E087
:100AF00040E05FE40E941A0988238CF020E030E097
:100B000040E05FE4C801B7010E94E8060E94D809EE
:100B10009B01AC01205030404040504806C0C80105
:100B2000B7010E94D8099B01AC01B901CA011F910C
:100B30000F91FF90EF900895A0E0B0E0E2EAF5E0B9
:100B40000C94580FDC012B01FA019C91923008F4AF
:100B500039C1EB018881823008F433C1943069F4E3
:100B6000843009F02FC111969C91119789819817B3
:100B700009F428C1A4E6B1E025C1843009F421C1FB
:100B80008230A9F4923009F01DC19A01AD0188E0CC
:100B9000EA010990AE01E90109929E018150C1F775
:100BA000E201898111969C918923818308C1923049
:100BB00009F407C112962D903C901397EB018A819E
:100BC0009B811496AD90BD90CD90DC901797EC80F2
:100BD000FD800E811F819101281B390BB90137FF60
:100BE00004C066277727621B730B603271050CF017
:100BF00061C0121613066CF537014801062E04C0B9
:100C000096948794779467940A94D2F721E030E021
:100C100040E050E004C0220F331F441F551F6A9567
:100C2000D2F721503040404050402E213F214023F8
:100C30005123211531054105510521F021E030E016
:100C400040E050E079018A01E628F72808291929AF
:100C50003CC0232BD1F1260E371E35014601062E4E
:100C600004C096948794779467940A94D2F721E00D
:100C700030E040E050E004C0220F331F441F551FF6
:100C80006A95D2F721503040404050402A213B2104
:100C90004C215D21211531054105510521F021E04F
:100CA00030E040E050E059016A01A628B728C82882
:100CB000D9280BC0821593052CF01C01AA24BB2453
:100CC000650103C0EE24FF24870111969C91D20197
:100CD00011968C91981709F445C0992339F0A80111
:100CE00097012A193B094C095D0906C0A601950127
:100CF0002E193F09400B510B57FD08C0118233825A
:100D0000228224833583468357831DC081E08183FB
:100D10003382228288279927DC01821B930BA40B44
:100D2000B50B84839583A683B7830DC0220F331F31
:100D3000441F551F248335834683578382819381C3
:100D40000197938382832481358146815781DA011B
:100D5000C9010197A109B1098F5F9F4FAF4FBF43F1
:100D600028F30BC0918333822282EA0CFB1C0C1DFA
:100D70001D1DE482F5820683178383E0808324812E
:100D800035814681578157FF1AC0C901AA2797FDAF
:100D9000A095BA2F81709070A070B070569547954D
:100DA00037952795822B932BA42BB52B8483958382
:100DB000A683B78382819381019693838283DF0127
:100DC00001C0D201CD01CDB7DEB7E2E10C94740FC2
:100DD000A0E2B0E0EEEEF6E00C94640F69837A8353
:100DE0008B839C832D833E834F835887E9E0EE2ECF
:100DF000F12CEC0EFD1EB701CE0101960E94C90B2D
:100E00008E010F5E1F4FB801CE0105960E94C90BDF
:100E10008A8991E089278A8BAE01475E5F4FB801CE
:100E2000C7010E949C050E94F40AA096E6E00C947B
:100E3000800FA0E2B0E0EFE1F7E00C94640F69836B
:100E40007A838B839C832D833E834F835887F9E07D
:100E5000EF2EF12CEC0EFD1EB701CE0101960E9483
:100E6000C90B8E010F5E1F4FB801CE0105960E947F
:100E7000C90BAE01475E5F4FB801C7010E949C05D8
:100E80000E94F40AA096E6E00C94800FA0E2B0E085
:100E9000ECE4F7E00C94580F69837A838B839C838E
:100EA0002D833E834F835887BE01675F7F4FCE01FE
:100EB00001960E94C90BBE016F5E7F4FCE01059661
:100EC0000E94C90B9985923088F089898230C8F0D8
:100ED000943019F4823051F404C0843029F49230F3
:100EE00081F484E691E0C6C0923049F420E09A850E
:100EF0008A89981321E02A87CE010996BBC08230E7
:100F000049F420E09A858A89981321E02A8BCE0142
:100F10004196B0C02D843E844F8458886D887E8869
:100F20008F88988CEE24FF248701AA24BB246501B6
:100F300040E050E060E070E0E0E0F0E0C10181708E
:100F40009070892BE9F0E60CF71C081D191D9A0119
:100F5000AB012A0D3B1D4C1D5D1D80E090E0A0E023
:100F6000B0E0E614F7040805190520F481E090E0EC
:100F7000A0E0B0E0BA01A901480F591F6A1F7B1F0A
:100F8000AA0CBB1CCC1CDD1C97FE08C081E090E0C5
:100F9000A0E0B0E0A82AB92ACA2ADB2A3196E032BA
:100FA000F10549F0660C771C881C991C56944794EF
:100FB00037942794C3CFFA85EA892B893C898B859E
:100FC0009C85280F391F2E5F3F4F17C0CA018170C3
:100FD0009070892B61F016950795F794E79480E05F
:100FE00090E0A0E0B0E8E82AF92A0A2B1B2B7695BE
:100FF0006795579547952F5F3F4F77FDE7CF0CC01B
:10100000440F551F661F771F17FD4160EE0CFF1C34
:10101000001F111F21503040403090E0590790E0F0
:10102000690790E4790760F32B8F3C8FDB01CA01DD
:101030008F779070A070B07080349105A105B105D4
:1010400061F447FD0AC0E114F1040105110529F01E
:10105000405C5F4F6F4F7F4F40781A8EFE1711F044
:1010600081E08A8F4D8F5E8F6F8F78A383E0898FA9
:10107000CE0149960E94F40AA096E2E10C94740F06
:10108000A8E1B0E0E6E4F8E00C94600F69837A83AD
:101090008B839C832D833E834F835887B9E0EB2E4F
:1010A000F12CEC0EFD1EB701CE0101960E94C90B7A
:1010B0008E010F5E1F4FB801CE0105960E94C90B2D
:1010C0002985223008F47CC03989323010F4B80107
:1010D0007AC08A859A8989278A87243011F022303C
:1010E00031F4231709F06CC064E671E06CC0343051
:1010F00039F41D861E861F86188A1C861B8604C02E
:10110000323021F484E08987B7015DC02B853C85AE
:101110008B899C89281B390B3C872B87ED84FE84A7
:101120000F851889AD88BE88CF88D88CEA14FB0457
:101130000C051D0540F4EE0CFF1C001F111F215073
:1011400030403C872B8720E030E040E050E080E0FA
:1011500090E0A0E0B0E46FE170E0EA14FB040C055D
:101160001D0540F0282B392B4A2B5B2BEA18FB0876
:101170000C091D09B695A79597958795EE0CFF1C50
:10118000001F111F6150704041F7DA01C9018F77CC
:101190009070A070B07080349105A105B10561F424
:1011A00027FD0AC0E114F1040105110529F0205CB6
:1011B0003F4F4F4F5F4F20782D873E874F87588B8B
:1011C000BE01675F7F4FCB010E94F40A6896EAE098
:1011D0000C947C0FA8E1B0E0E0EFF8E00C94640F11
:1011E00069837A838B839C832D833E834F835887C7
:1011F00089E0E82EF12CEC0EFD1EB701CE01019620
:101200000E94C90B8E010F5E1F4FB801CE010596DB
:101210000E94C90B8985823040F08989823028F08C
:10122000B801C7010E94410C01C08FEF6896E6E04B
:101230000C94800FA8E1B0E0E0E2F9E00C94640FB8
:1012400069837A838B839C832D833E834F83588766
:1012500089E0E82EF12CEC0EFD1EB701CE010196BF
:101260000E94C90B8E010F5E1F4FB801CE0105967B
:101270000E94C90B8985823040F08989823028F02C
:10128000B801C7010E94410C01C08FEF6896E6E0EB
:101290000C94800FA8E1B0E0E0E5F9E00C94640F55
:1012A00069837A838B839C832D833E834F83588706
:1012B00089E0E82EF12CEC0EFD1EB701CE0101965F
:1012C0000E94C90B8E010F5E1F4FB801CE0105961B
:1012D0000E94C90B8985823040F08989823028F0CC
:1012E000B801C7010E94410C01C081E06896E6E0A8
:1012F0000C94800FA8E0B0E0E0E8F9E00C94610FF6
:101300009B01AC0183E08983DA01C9018827B7FD1D
:1013100083959927AA27BB27B82E211531054105AA
:10132000510519F482E089833AC08823A9F020305E
:1013300080E0380780E0480780E8580729F460E03B
:1013400070E080E09FEC30C0EE24FF248701E21AB9
:10135000F30A040B150B02C079018A018EE1C82E35
:10136000D12CDC82CB82ED82FE820F831887C801EC
:10137000B7010E94A50A01971816190684F4082ED1
:1013800004C0EE0CFF1C001F111F0A94D2F7ED825F
:10139000FE820F831887C81AD90ADC82CB82BA82F0
:1013A000CE0101960E94F40A2896E9E00C947D0F84
:1013B000ACE0B0E0EEEDF9E00C94680F69837A835D
:1013C0008B839C83BE016B5F7F4FCE0101960E9491
:1013D000C90B8D81823061F1823050F1843021F46B
:1013E0008E81882351F12EC02F81388537FD20C092
:1013F0006E812F3131051CF06623F9F023C08EE198
:1014000090E0821B930B29853A854B855C8504C04F
:1014100056954795379527958A95D2F76623B1F06B
:1014200050954095309521953F4F4F4F5F4F0EC0DF
:1014300020E030E040E050E009C02FEF3FEF4FEFF9
:101440005FE704C020E030E040E050E8B901CA01A5
:101450002C96E2E00C94840FA8E0B0E0E2E3FAE01E
:101460000C94620F7B018C0161157105810591055A
:1014700019F482E0898360C083E089838EE1C82EFD
:10148000D12CDC82CB82ED82FE820F831887C801CB
:10149000B7010E94A50ABC016150704077FF39C0B6
:1014A000EE27FF27E61BF70B20E030E040E050E09E
:1014B00081E090E0A0E0B0E00E2E04C0880F991FFC
:1014C000AA1FBB1F0A94D2F70197A109B1098E2167
:1014D0009F21A023B1230097A105B10521F021E0B0
:1014E00030E040E050E004C016950795F794E7948B
:1014F000EA95D2F72E293F29402B512B2D833E838D
:101500004F8358878EE190E0861B970B9C838B83DB
:1015100013C06115710581F0062E04C0EE0CFF1C8E
:10152000001F111F0A94D2F7ED82FE820F831887E5
:10153000C61AD70ADC82CB821A82CE0101960E949B
:10154000F40A2896E8E00C947E0FEF92FF920F9336
:101550001F937B018C0180E0E81680E0F80681E0B3
:10156000080780E0180788F48FEFE816F1040105FA
:10157000110531F028F088E090E0A0E0B0E017C05D
:1015800080E090E0A0E0B0E012C080E0E81680E0EB
:10159000F80680E0080781E0180728F088E190E06D
:1015A000A0E0B0E004C080E190E0A0E0B0E020E284
:1015B00030E040E050E0281B390B4A0B5B0B04C0C5
:1015C00016950795F794E7948A95D2F7F701E459B1
:1015D000FE4F8081281B310941095109C9011F9122
:1015E0000F91FF90EF900895DF92EF92FF920F938B
:1015F0001F93FC01E480F58006811781D1808081F2
:10160000823048F480E090E0A0E1B0E0E82AF92AD6
:101610000A2B1B2BA5C0843009F49FC0823021F413
:10162000EE24FF24870105C0E114F1040105110532
:1016300019F4E0E0F0E096C0628173819FEF6238B8
:1016400079070CF05BC022E83FEF261B370B2A31ED
:1016500031052CF020E030E040E050E02AC0B80135
:10166000A701022E04C076956795579547950A9471
:10167000D2F781E090E0A0E0B0E004C0880F991FAD
:10168000AA1FBB1F2A95D2F70197A109B1098E2184
:101690009F21A023B1230097A105B10521F081E08E
:1016A00090E0A0E0B0E09A01AB01282B392B4A2B47
:1016B0005B2BDA01C9018F779070A070B070803415
:1016C0009105A105B10539F427FF09C0205C3F4F02
:1016D0004F4F5F4F04C0215C3F4F4F4F5F4FE0E0E3
:1016E000F0E02030A0E03A07A0E04A07A0E45A0763
:1016F00010F0E1E0F0E079018A0127C0603871055F
:1017000064F5FB01E158FF4FD801C7018F77907056
:10171000A070B07080349105A105B10539F4E7FEE1
:101720000DC080E490E0A0E0B0E004C08FE390E062
:10173000A0E0B0E0E80EF91E0A1F1B1F17FF05C04E
:1017400016950795F794E794319687E016950795D7
:10175000F794E7948A95D1F705C0EE24FF2487011A
:10176000EFEFF0E06E2F679566276795902F9F77D4
:10177000D794DD24D7948E2F8695492F462B582F4A
:101780005D29B701CA011F910F91FF90EF90DF9083
:101790000895FC01DB01408151812281622F6F7726
:1017A00070E0221F2227221F9381892F880F822B0E
:1017B000282F30E0991F9927991F11969C93119714
:1017C00021153105A9F5411551056105710511F482
:1017D00082E037C082E89FEF13969C938E93129716
:1017E0009A01AB0167E0220F331F441F551F6A9512
:1017F000D1F783E08C930DC0220F331F441F551F78
:1018000012968D919C911397019713969C938E93AA
:101810001297203080E0380780E0480780E45807BE
:1018200058F314962D933D934D935C931797089519
:101830002F3F310579F4411551056105710519F402
:1018400084E08C93089564FF03C081E08C9312C000
:101850001C9210C02F57304013963C932E93129732
:1018600083E08C9387E0440F551F661F771F8A958E
:10187000D1F7706414964D935D936D937C93179795
:1018800008951F93DC01FB019C91923008F447C03E
:101890008081823008F443C0943051F411961C9139
:1018A000843099F58181682F70E0611B71093FC018
:1018B000843021F0923031F48230B9F18181882373
:1018C00089F12DC011961C9111978230F1F0818120
:1018D0001817D9F412962D913C9113978281938118
:1018E0008217930794F028173907BCF014968D914E
:1018F0009D910D90BC91A02D248135814681578109
:10190000281739074A075B0718F4112341F00AC06A
:1019100082179307A407B50740F4112319F061E07B
:1019200070E005C06FEF7FEF02C060E070E0CB01B8
:101930001F910895FB01DC018D9101908019011028
:10194000D9F3990B0895FB01DC0101900D92002061
:10195000E1F70895AEE0B0E0E0EBFCE00C94660F38
:101960000D891E8986E08C831A8309838FEF9FE798
:101970009E838D83CE014996AC016F89788DCE010F
:1019800001960E94CD0C2F813885020F131FF8019C
:1019900010822E96E4E00C94820FABE0B0E0E3ED11
:1019A000FCE00C94580F3C012B015A01FC011782FA
:1019B0001682838181FD03C06FEF7FEFC8C19AE07B
:1019C000892E1E010894211C311CF3012381F20190
:1019D00023FD859123FF81912F01882309F4B4C150
:1019E000853239F423FD859123FF81912F018532C2
:1019F00029F4B30190E00E94C20EE7CF982FDD24B6
:101A0000CC249924FFE1FD15D0F09B3269F09C3283
:101A100028F4903259F0933291F40EC09D3249F07F
:101A2000903369F441E024C052E0D52A84E0D82AFA
:101A300028C098E0D92A25C0E0E1DE2A22C0D7FCE0
:101A400029C0892F80538A3070F4D6FE05C0989C37
:101A5000902C1124980E15C0C89CC02C1124C80EBF
:101A6000F0E2DF2A0EC09E3229F4D6FC6DC140E4BC
:101A7000D42A07C09C3619F450E8D52A02C09836FB
:101A800049F4F20123FD959123FF91912F019923B0
:101A900009F0B8CF892F8554833018F080528330F5
:101AA00038F444E050E0A40EB51E5FE359830FC044
:101AB000933631F0933779F0933509F056C020C052
:101AC000F5018081898342E050E0A40EB51E7101CA
:101AD00001E010E012C0F501E080F180D6FC03C007
:101AE0006FEF7FEF02C0692D70E042E050E0A40E7E
:101AF000B51EC7010E94B70E8C015FE7D52214C046
:101B0000F501E080F180D6FC03C06FEF7FEF02C0EB
:101B1000692D70E042E050E0A40EB51EC7010E949E
:101B2000AC0E8C0150E8D52AD3FE07C01AC0B30111
:101B300080E290E00E94C20ECA948C2D90E00817BB
:101B40001907A8F30EC0F701D7FC8591D7FE819144
:101B50007F01B30190E00E94C20EC110CA940150EF
:101B600010400115110579F7ECC0943611F0993643
:101B700071F5D7FE08C0F501E080F1800281138184
:101B800044E050E00AC0F501808191817C0100278A
:101B9000F7FC0095102F42E050E0A40EB51E5FE662
:101BA000D52217FF0AC010950095F094E094E11C2F
:101BB000F11C011D111D80E8D82A2AE030E0A101A6
:101BC000C801B7010E94EE0EF82EF21840C09537FA
:101BD00029F41D2D1F7E2AE030E01DC01D2D197F28
:101BE0009F3661F0903720F4983509F0ADC00FC0F2
:101BF000903739F0983709F0A7C004C028E030E0EA
:101C00000AC0106114FD146020E130E004C014FD2E
:101C1000166020E132E017FF08C0F5016081718194
:101C20008281938144E050E008C0F5018081918178
:101C3000BC0180E090E042E050E0A40EB51EA1019E
:101C40000E94EE0EF82EF2188FE7D82ED122D6FE83
:101C50000BC05EEFD522F91438F4D4FE07C0D2FCD5
:101C600005C08FEED82202C01F2D01C0192DD4FE51
:101C70000DC0FE01EF0DF11D8081803319F499EE46
:101C8000D92208C01F5FD2FE05C003C08D2D867803
:101C900009F01F5F0D2DD3FC14C0D0FE0FC01C1522
:101CA00010F09F2C0BC09F2C9C0C911A1C2D06C071
:101CB000B30180E290E00E94C20E1F5F1C15C0F3CA
:101CC00004C01C1510F4C11A01C0CC2404FF10C0BC
:101CD000B30180E390E00E94C20E02FF1EC001FD2E
:101CE00003C088E790E002C088E590E0B3010CC033
:101CF000802F867891F001FF02C08BE201C080E264
:101D0000D7FC8DE2B30190E00E94C20E06C0B30181
:101D100080E390E00E94C20E9A94F914C0F3FA9402
:101D2000F101EF0DF11DB301808190E00E94C20E20
:101D3000FF20A9F706C0B30180E290E00E94C20E26
:101D4000CA94CC20C1F741CEF30166817781CB01E3
:101D50002B96E2E10C94740FFC01059061507040E9
:101D60000110D8F7809590958E0F9F1F0895FC0164
:101D70006150704001900110D8F7809590958E0FBA
:101D80009F1F08950F931F93CF93DF938C01EB0157
:101D90008B8181FF1BC082FF0DC02E813F818C8112
:101DA0009D812817390764F4E881F9810193F9834B
:101DB000E88306C0E885F985802F0995892B31F4E1
:101DC0008E819F8101969F838E8302C00FEF1FEF4C
:101DD000C801DF91CF911F910F910895FA01AA27B1
:101DE000283051F1203181F1E8946F936E7F6E5F5E
:101DF0007F4F8F4F9F4FAF4FB1E03ED0B4E03CD00C
:101E0000670F781F891F9A1FA11D680F791F8A1FEE
:101E1000911DA11D6A0F711D811D911DA11D20D055
:101E200009F468943F912AE0269F11243019305D0F
:101E30003193DEF6CF010895462F4770405D419300
:101E4000B3E00FD0C9F7F6CF462F4F70405D4A334D
:101E500018F0495D31FD4052419302D0A9F7EACF15
:101E6000B4E0A6959795879577956795BA95C9F744
:101E700000976105710508959B01AC010A2E069437
:101E80005795479537952795BA95C9F7620F731FF0
:101E9000841F951FA01D0895991B79E004C0991F08
:101EA000961708F0961B881F7A95C9F780950895B4
:101EB0002F923F924F925F926F927F928F929F925A
:101EC000AF92BF92CF92DF92EF92FF920F931F9348
:101ED000CF93DF93CDB7DEB7CA1BDB0B0FB6F894F9
:101EE000DEBF0FBECDBF09942A88398848885F8439
:101EF0006E847D848C849B84AA84B984C884DF80AA
:101F0000EE80FD800C811B81AA81B981CE0FD11D8D
:101F10000FB6F894DEBF0FBECDBFED010895F89463
:021F2000FFCFF1
:101F2200205A6164656A2050494E2061202A2000AF
:101F320020202020202020202020202020202000BF
:101F42003132333400202020202020202020202065
:101F5200202020202000256400505249535455501F
:101F620020504F564F4C454E210050524953545524
:101F720050204F44455052454E2100303030300001
:101F82000A00FFFF00000000000000000001020242
:101F920003030303040404040404040405050505FF
:101FA20005050505050505050505050506060606DB
:101FB20006060606060606060606060606060606BF
:101FC20006060606060606060606060607070707AB
:101FD200070707070707070707070707070707078F
:101FE200070707070707070707070707070707077F
:101FF200070707070707070707070707070707076F
:10200200070707070707070707070707080808085A
:10201200080808080808080808080808080808083E
:10202200080808080808080808080808080808082E
:10203200080808080808080808080808080808081E
:10204200080808080808080808080808080808080E
:1020520008080808080808080808080808080808FE
:1020620008080808080808080808080808080808EE
:1020720008080808080808080808080808080808DE
:0C208200080808080808080808080808F2
:00000001FF
